:100000008FC00000A8C00000A6C00000A4C000006F
:10001000A2C00000A0C000009EC000009CC0000064
:100020009AC0000098C0000096C00000A3C4000061
:1000300092C0000090C000008EC000008CC0000084
:100040008AC0000088C0000086C0000084C0000094
:1000500082C0000080C000007EC000007CC00000A4
:100060007AC0000078C0000076C0000074C00000B4
:1000700072C0000005010904A1010901A1000501E8
:1000800009300931159C256475089502818205099E
:100090000902090115002501750195028102750605
:1000A00095018101C0C01201100100000008EB039E
:1000B000432000000102000109022200010100C0EA
:1000C00032090400000103000000092111010001B0
:1000D0002232000705810308000A040309041803FB
:1000E0004400650061006E002000430061006D0067
:1000F000650072006100000026034C0055004600B8
:10010000410020004A006F0079007300740069000C
:1001100063006B002000440065006D006F0000006C
:1001200011241FBECFEFD2E0DEBFCDBF11E0A0E0B3
:10013000B1E0EAEDFEE002C005900D92AC30B107EF
:10014000D9F711E0ACE0B1E001C01D92AC31B107CC
:10015000E1F78DD0C0C654CFFB01DC0104C08D9106
:100160000190801921F441505040C8F7881B990B29
:100170000895FB01DC0102C001900D9241505040F6
:10018000D8F70895DC0101C06D9341505040E0F76D
:10019000089585B18F70806685B9089585B18F7097
:1001A000806185B90895D901FA0189B129B1809595
:1001B0008F71982F83FF02C08CE903C081FF02C0BA
:1001C00084E6818390FF02C084E603C092FF02C0F0
:1001D0008CE9808394FF02C082E0828327FD03C004
:1001E00082818160828383E090E08D939C9380E0A4
:1001F0000895089580E091E075C480E091E05CC5C9
:1002000085B18F70806A85B980E091E02DD5882313
:1002100021F485B18F70806585B98091E20084609A
:100220008093E200089584B7877F84BF88E10FB68A
:10023000F89480936000109260000FBE80E090E020
:1002400020E80FB6F89420936100809361000FBE00
:100250008AB1807E8AB98BB18F618BB984B1806F8E
:1002600084B985B18F7085B957985F9A76C3DBDF03
:1002700085B18F70806185B980E091E03CD41FD456
:10028000FBCFDA019330B1F0943028F4913041F093
:10029000923079F50AC0913211F1923251F524C0B1
:1002A000E6EAF0E022E130E028C0E8EBF0E022E20C
:1002B00030E023C0813049F0813018F08230C9F439
:1002C0000AC0EAEDF0E0849103C0EEEDF0E0849125
:1002D000282F30E012C0E8EFF0E08491F9CFEAEC8B
:1002E000F0E029E030E009C0E4E7F0E022E330E0AC
:1002F00004C0E0E0F0E020E030E0ED93FC93C901C1
:100300000895DF93CF9300D0CDB7DEB7E4E1F1E0FD
:100310008091F100819381E0EC31F807C9F7809179
:10032000140130911501353009F49FC0363048F47E
:10033000313009F44BC0313070F0333009F021C155
:1003400045C0383009F4D6C0393009F4FBC0363026
:1003500009F017C1B4C0803821F0823809F011C10A
:1003600008C090910F0180911001882391F0926054
:1003700010C0809118018093E9008091EB0090E01B
:1003800025E0969587952A95E1F7982F9170109220
:10039000E9008091E800877F8093E8009093F10066
:1003A0001092F1008091E800982F9E7F9093E800D2
:1003B0008F778093E80005C080911301882309F4AA
:1003C000E1C08091E80082FFF7CFB2C0882319F026
:1003D000823009F0D6C090E08F719070009719F0CC
:1003E0000297B9F50CC080911601813009F0CAC09E
:1003F00010921001333069F5809310012AC080916A
:100400001601882331F520911801277009F4BAC02C
:100410002093E9008091EB0080FF1BC03130A1F4F4
:100420008091EB0080618093EB0081E090E002C05E
:10043000880F991F2A95E2F78093EA001092EA004C
:100440008091EB00886003C08091EB008062809314
:10045000EB001092E9008091E800877F8093E8002C
:100460008091E800982F9E7F67C0882309F089C09B
:10047000209116018091E800877F8093E8008091A9
:10048000E800982F9E7F9093E8008F778093E80094
:1004900005C080911301882309F474C08091E8009D
:1004A00080FFF7CF922F9F77892F80688093E3009A
:1004B000992309F467C083E08093130163C08058D7
:1004C000823008F05EC08091160190911701609112
:1004D0001801AE014F5F5F4FD4DEBC01009709F4F5
:1004E00051C08091E800877F8093E80089819A81DC
:1004F00073D11EC0803809F044C08091E800877F26
:100500008093E800809111018093F1008091E800D0
:10051000982F9E7F9093E8008F778093E80004C027
:1005200080911301882371F18091E80082FFF8CF58
:100530008091E800982F9B7F9093E8008F778093BD
:10054000E80020C08823E9F4209116012230D0F47D
:100550008091E800877F8093E800209311018091CB
:10056000E800982F9E7F9093E8008F778093E800B3
:10057000222311F084E001C083E08093130140DE68
:1005800001C03BDE8091E80083FF0AC08091EB0050
:1005900080628093EB008091E800877F8093E80081
:1005A0000F900F90CF91DF91089528E030E040E068
:1005B00003C04F5F220F331F28173907D0F3842F52
:1005C0008295807F08958093E9008091EB0081609F
:1005D0008093EB001092ED006093EC004093ED00EF
:1005E0008091EE00881F8827881F08951092F400DC
:1005F00090E09093E9001092F0001092E800809152
:10060000ED008D7F8093ED008091EB008E7F8093D5
:10061000EB009F5F953069F708958091140188235E
:10062000BCF404C0809113018823F9F08091E800A4
:1006300082FFF8CF8091E800982F9B7F9093E8008D
:100640008F778093E800089580911301882369F0E3
:100650008091E80080FFF8CF8091E800982F9E7F7E
:100660009093E8008F778093E800089594E6809156
:10067000EC0080FF05C08091E80080FF05C01FC02E
:100680008091E80082FD1BC080911301882311F442
:1006900082E008958091EB0085FF02C081E008951B
:1006A0008091E10082FFE3CF8091E1008B7F809316
:1006B000E100992311F483E008959150D8CF80E0B0
:1006C0000895DF92EF92FF920F931F93CF93DF93E2
:1006D000182F092FEB017A01C9DFD82E882339F5AD
:1006E000812F902F9C01890120C08091E80085FD19
:1006F00016C08091E800982F9E7F9093E8008F7736
:100700008093E800E114F10431F0F701099581309C
:1007100011F484E00DC0AADF882339F009C0F80184
:1007200081918F018093F10021972097F1F68D2D13
:10073000DF91CF911F910F91FF90EF90DF9008957F
:10074000FC0140911A0150911B019B01461757076C
:1007500008F49A0140E02EC08091E80083FF02C0B7
:1007600081E008958091E80082FD2EC08091130100
:10077000882381F18091E80080FF1CC005C0819131
:100780008093F100215030402115310521F08091F6
:10079000F2008830A0F38091F20040E0883009F444
:1007A00041E08091E800982F9E7F9093E8008F773A
:1007B0008093E8002115310579F6442369F604C0D9
:1007C00080911301882331F08091E80082FFF8CFF7
:1007D00080E0089582E00895DC0140911A01509173
:1007E0001B019B014617570708F49A0140E030C0EF
:1007F0008091E80083FF02C081E008958091E800C5
:1008000082FD30C080911301882391F18091E8002E
:1008100080FF1EC007C0FD011196E491E093F10036
:10082000215030402115310521F08091F2008830AF
:1008300090F38091F20040E0883009F441E080912B
:10084000E800982F9E7F9093E8008F778093E800D0
:100850002115310569F6442359F604C0809113012E
:10086000882331F08091E80082FFF8CF80E008957E
:1008700082E00895FC0122C08091E80083FF02C05D
:1008800081E0089580911301882331F18091E8007F
:1008900082FFF2CF06C08091F100819361507040D9
:1008A00021F08091F2008823B1F78091E800982F21
:1008B0009B7F9093E8008F778093E8006115710526
:1008C000D9F604C080911301882331F08091E800AB
:1008D00080FFF8CF80E0089582E0089545D047D0AA
:1008E00010921301109211011092100110920F0139
:1008F00084E089BD89B5826089BD09B400FEFDCF61
:100900008091D800982F9F779093D800806880932B
:10091000D800809163008E7F809363008091D8001F
:100920008F7D8093D8008091E0008E7F8093E000DF
:100930008091E1008E7F8093E1008091E2008160F0
:100940008093E2008091E100877F8093E1008091B5
:10095000E20088608093E2000895C0DF81E0809328
:1009600012017894089508951092E200089510926B
:10097000E10008951F920F920FB60F9211242F934A
:100980003F934F935F936F937F938F939F93AF9317
:10099000BF93EF93FF938091E10080FF1CC0809193
:1009A000E20080FF18C08091E1008E7F8093E1001B
:1009B0008091E2008E7F8093E2008091E20080616E
:1009C0008093E2008091D80080628093D80019BCA7
:1009D00010921301E3DB8091E10084FF2AC0809133
:1009E000E20084FF26C084E089BD89B5826089BDAC
:1009F00009B400FEFDCF8091D8008F7D8093D80090
:100A00008091E1008F7E8093E1008091E2008F7EF3
:100A10008093E2008091E20081608093E200809107
:100A20001101882311F481E001C084E08093130157
:100A3000B0DB8091E10083FF23C08091E20083FF5F
:100A40001FC08091E100877F8093E10082E0809366
:100A50001301109211018091E1008E7F8093E100DB
:100A60008091E2008E7F8093E2008091E2008061BD
:100A70008093E200BBDD80E060E042E0A4DD73DF54
:100A80008091E10082FF0AC08091E20082FF06C0EF
:100A90008091E1008B7F8093E100ACDBFF91EF91CF
:100AA000BF91AF919F918F917F916F915F914F9186
:100AB0003F912F910F900FBE0F901F9018951F938D
:100AC00080911301882361F01091E9001092E900F0
:100AD0008091E80083FF01C014DC17701093E900D7
:100AE0001F910895FC0182859385009719F0019765
:100AF0009387828708952F923F924F925F926F92D1
:100B00007F928F929F92AF92BF92CF92DF92EF929D
:100B1000FF920F931F93DF93CF9300D000D0CDB7F8
:100B2000DEB77C012DB63EB680911301843009F00A
:100B30007FC0F70181818093E9008091E80085FF03
:100B400077C04DB6FEB7FC83F70146818DB79EB7DF
:100B5000841B91090FB6F8949EBF0FBE8DBF0DB7D1
:100B60001EB70F5F1F4F19821B821A82602E512EF3
:100B7000C80160E070E050E005DBC701BE016F5FB7
:100B80007F4FA8019E012E5F3F4F0DDB782EF701AE
:100B9000B480A5809A808B80C8016B2D7A2D492D59
:100BA000582DDADA8C01F70180859185892B19F4AB
:100BB000CC24DD240BC020E0F70182859385892BAE
:100BC00009F021E081E02827C22EDD248B2D9A2D0B
:100BD000662D752D492D582DCCDA6A817B816115E2
:100BE0007105F1F0772021F4012B11F4CD28C1F02B
:100BF000F70180859185938782878981882311F009
:100C00008093F100862D952D40E050E05ADD8091D3
:100C1000E800982F9E7F9093E8008F778093E800FC
:100C2000842D9C819C010FB6F8943EBF0FBE2DBF52
:100C30000FB6F8943EBE0FBE2DBE0F900F900F90D2
:100C40000F90CF91DF911F910F91FF90EF90DF9068
:100C5000CF90BF90AF909F908F907F906F905F905C
:100C60004F903F902F9008951F93CF93DF93DC0117
:100C70000796FC0185E0EF0119928A95E9F781E07A
:100C800017968C93179784EF91E019969C938E9307
:100C9000189711961C91119712968D919C9113970C
:100CA00084DC482F4260812F61EC8DDC811181E072
:100CB000DF91CF911F9108956F927F928F929F92B3
:100CC000BF92CF92DF92EF92FF920F931F93DF9329
:100CD000CF9300D00F92CDB7DEB74C016DB67EB684
:100CE0008091E80083FFE1C0F401808190E02091D1
:100CF0001801309119012817390709F0D6C08091E1
:100D00001501833009F47CC0843030F4813071F0F7
:100D1000823009F0CAC0ADC08A3009F493C08B306C
:100D200009F47BC0893009F0C0C032C08091140141
:100D3000813A09F0BAC08091E800877F8093E8008B
:100D40001B821A82809116018983F4014681848175
:100D5000958160E070E050E015DAF401448155813E
:100D6000C401BE016F5F7F4F9E012E5F3F4F1BDAB4
:100D70006A817B81F40184819581E2DC8091E800C5
:100D8000982F9B7F9093E8008F778093E8008DC029
:100D900080911401813209F088C0BEB68091E800CC
:100DA000877F8093E800E0901A01F0901B018DB7D7
:100DB0009EB78E199F090FB6F8949EBF0FBE8DBFC8
:100DC0000DB71EB70F5F1F4FD0901601C801B701B6
:100DD00051DD8091E800982F9E7F9093E8008F77F7
:100DE0008093E800C4016D2DA801970102DA262D39
:100DF0003B2DC9010FB6F8949EBF0FBE8DBF55C0E5
:100E000080911401813A09F050C08091E800877FF9
:100E10008093E800F40187813CC080911401813205
:100E200009F043C08091E800877F8093E80020E0CC
:100E30008091160190911701892B09F021E0F401AE
:100E4000278332C080911401813279F58091E800C6
:100E5000877F8093E8008091160190911701807040
:100E600036E0969587953A95E1F7F401918780876A
:100E70001BC080911401813AC1F48091E800877F02
:100E80008093E800F40180859185969587959695E5
:100E900087958093F1008091E800982F9E7F909332
:100EA000E8008F778093E800B8DB0FB6F8947EBE39
:100EB0000FBE6DBE0F900F900F90CF91DF911F91DD
:100EC0000F91FF90EF90DF90CF90BF909F908F9009
:0A0ED0007F906F900895F894FFCF13
:0C0EDA00000108000C01030000000000F3
:00000001FF
